:020000040000fa
:080000000002040000000000f2
:020000040000fa
:040008009a03000057
:020000040000fa
:04000c00b403000039
:020000040000fa
:040010006603000083
:020000040000fa
:04001400ce03000017
:020000040000fa
:04001800e8030000f9
:020000040000fa
:04001c0032030000ab
:020000040000fa
:040020008003000059
:020000040000fa
:040024004c03000089
:020000040000fa
:040028003c04000094
:020000040000fa
:04002c003c04000090
:020000040000fa
:040030003c0400008c
:020000040000fa
:040034003c04000088
:020000040000fa
:040038003c04000084
:020000040000fa
:04003c003c04000080
:020000040000fa
:040040003c0400007c
:020000040000fa
:040044003c04000078
:020000040000fa
:040048003c04000074
:020000040000fa
:04004c003c04000070
:020000040000fa
:040050003c0400006c
:020000040000fa
:040054003c04000068
:020000040000fa
:040058003c04000064
:020000040000fa
:04005c003c04000060
:020000040000fa
:040060003c0400005c
:020000040000fa
:040064003c04000058
:020000040000fa
:040068003c04000054
:020000040000fa
:04006c003c04000050
:020000040000fa
:040070003c0400004c
:020000040000fa
:040074003c04000048
:020000040000fa
:040078003c04000044
:020000040000fa
:04007c003c04000040
:020000040000fa
:040080003c0400003c
:020000040000fa
:040084003c04000038
:020000040000fa
:040088003c04000034
:020000040000fa
:04008c003c04000030
:020000040000fa
:040090003c0400002c
:020000040000fa
:040094003c04000028
:020000040000fa
:040098003c04000024
:020000040000fa
:04009c003c04000020
:020000040000fa
:0400a0003c0400001c
:020000040000fa
:0400a4003c04000018
:020000040000fa
:0400a8003c04000014
:020000040000fa
:0400ac003c04000010
:020000040000fa
:0400b0003c0400000c
:020000040000fa
:0400b4003c04000008
:020000040000fa
:0400b8003c04000004
:020000040000fa
:0400bc003c04000000
:020000040000fa
:0400c0003c040000fc
:020000040000fa
:0400c4003c040000f8
:020000040000fa
:0400c8003c040000f4
:020000040000fa
:0400cc003c040000f0
:020000040000fa
:0400d0003c040000ec
:020000040000fa
:0400d4003c040000e8
:020000040000fa
:0400d8003c040000e4
:020000040000fa
:0400dc003c040000e0
:020000040000fa
:0400e0003c040000dc
:020000040000fa
:0400e4003c040000d8
:020000040000fa
:0400e8003c040000d4
:020000040000fa
:0400ec003c040000d0
:020000040000fa
:0400f0003c040000cc
:020000040000fa
:0400f4003c040000c8
:020000040000fa
:0400f8003c040000c4
:020000040000fa
:0400fc003c040000c0
:020000040000fa
:040100003c040000bb
:020000040000fa
:040104003c040000b7
:020000040000fa
:040108003c040000b3
:020000040000fa
:04010c003c040000af
:020000040000fa
:040110003c040000ab
:020000040000fa
:040114003c040000a7
:020000040000fa
:040118003c040000a3
:020000040000fa
:04011c003c0400009f
:020000040000fa
:040120003c0400009b
:020000040000fa
:040124003c04000097
:020000040000fa
:040128003c04000093
:020000040000fa
:04012c003c0400008f
:020000040000fa
:040130003c0400008b
:020000040000fa
:040134003c04000087
:020000040000fa
:040138003c04000083
:020000040000fa
:04013c003c0400007f
:020000040000fa
:040140003c0400007b
:020000040000fa
:040144003c04000077
:020000040000fa
:040148003c04000073
:020000040000fa
:04014c003c0400006f
:020000040000fa
:040150003c0400006b
:020000040000fa
:040154003c04000067
:020000040000fa
:040158003c04000063
:020000040000fa
:04015c003c0400005f
:020000040000fa
:040160003c0400005b
:020000040000fa
:040164003c04000057
:020000040000fa
:040168003c04000053
:020000040000fa
:04016c003c0400004f
:020000040000fa
:040170003c0400004b
:020000040000fa
:040174003c04000047
:020000040000fa
:040178003c04000043
:020000040000fa
:04017c003c0400003f
:020000040000fa
:040180003c0400003b
:020000040000fa
:040184003c04000037
:020000040000fa
:040188003c04000033
:020000040000fa
:04018c003c0400002f
:020000040000fa
:040190003c0400002b
:020000040000fa
:040194003c04000027
:020000040000fa
:04019800020400005d
:020000040000fa
:04019c003c0400001f
:020000040000fa
:0401a0003c0400001b
:020000040000fa
:0401a4003c04000017
:020000040000fa
:0401a8003c04000013
:020000040000fa
:0401ac003c0400000f
:020000040000fa
:0401b0003c0400000b
:020000040000fa
:0401b4003c04000007
:020000040000fa
:0401b8003c04000003
:020000040000fa
:0401bc003c040000ff
:020000040000fa
:0401c0003c040000fb
:020000040000fa
:0401c4003c040000f7
:020000040000fa
:0401c8003c040000f3
:020000040000fa
:0401cc003c040000ef
:020000040000fa
:0401d0003c040000eb
:020000040000fa
:0401d4003c040000e7
:020000040000fa
:0401d8003c040000e3
:020000040000fa
:0401dc003c040000df
:020000040000fa
:0401e0003c040000db
:020000040000fa
:0401e4003c040000d7
:020000040000fa
:0401e8003c040000d3
:020000040000fa
:0401ec003c040000cf
:020000040000fa
:0401f0003c040000cb
:020000040000fa
:0401f4003c040000c7
:020000040000fa
:0401f8003c040000c3
:020000040000fa
:0401fc003c040000bf
:020000040000fa
:040200003c040000ba
:020000040000fa
:040204003c040000b6
:020000040000fa
:040208003c040000b2
:020000040000fa
:04020c003c040000ae
:020000040000fa
:040210003c040000aa
:020000040000fa
:040214003c040000a6
:020000040000fa
:040218003c040000a2
:020000040000fa
:04021c003c0400009e
:020000040000fa
:040220003c0400009a
:020000040000fa
:040224003c04000096
:020000040000fa
:040228003c04000092
:020000040000fa
:04022c003c0400008e
:020000040000fa
:040230003c0400008a
:020000040000fa
:040234003c04000086
:020000040000fa
:040238003c04000082
:020000040000fa
:04023c003c0400007e
:020000040000fa
:040240003c0400007a
:020000040000fa
:040244003c04000076
:020000040000fa
:040248003c04000072
:020000040000fa
:04024c003c0400006e
:020000040000fa
:040250003c0400006a
:020000040000fa
:040254003c04000066
:020000040000fa
:040258003c04000062
:020000040000fa
:04025c003c0400005e
:020000040000fa
:040260003c0400005a
:020000040000fa
:040264003c04000056
:020000040000fa
:040268003c04000052
:020000040000fa
:04026c003c0400004e
:020000040000fa
:040270003c0400004a
:020000040000fa
:040274003c04000046
:020000040000fa
:040278003c04000042
:020000040000fa
:04027c003c0400003e
:020000040000fa
:040280003c0400003a
:020000040000fa
:040284003c04000036
:020000040000fa
:040288003c04000032
:020000040000fa
:04028c003c0400002e
:020000040000fa
:040290003c0400002a
:020000040000fa
:040294003c04000026
:020000040000fa
:040298003c04000022
:020000040000fa
:04029c003c0400001e
:020000040000fa
:0402a0003c0400001a
:020000040000fa
:0402a4003c04000016
:020000040000fa
:0402a8003c04000012
:020000040000fa
:0402ac003c0400000e
:020000040000fa
:0402b0003c0400000a
:020000040000fa
:0402b4003c04000006
:020000040000fa
:0402b8003c04000002
:020000040000fa
:0402bc003c040000fe
:020000040000fa
:0402c0003c040000fa
:020000040000fa
:0402c4003c040000f6
:020000040000fa
:0402c8003c040000f2
:020000040000fa
:0402cc003c040000ee
:020000040000fa
:0402d0003c040000ea
:020000040000fa
:0402d4003c040000e6
:020000040000fa
:0402d8003c040000e2
:020000040000fa
:0402dc003c040000de
:020000040000fa
:0402e0003c040000da
:020000040000fa
:0402e4003c040000d6
:020000040000fa
:0402e8003c040000d2
:020000040000fa
:0402ec003c040000ce
:020000040000fa
:0402f0003c040000ca
:020000040000fa
:0402f4003c040000c6
:020000040000fa
:0402f8003c040000c2
:020000040000fa
:0402fc003c040000be
:020000040000fa
:040300003c040000b9
:020000040000fa
:040304003c040000b5
:020000040000fa
:040308003c040000b1
:020000040000fa
:04030c003c040000ad
:020000040000fa
:040310003c040000a9
:020000040000fa
:040314003c040000a5
:020000040000fa
:040318003c040000a1
:020000040000fa
:04031c003c0400009d
:020000040000fa
:040320003c04000099
:020000040000fa
:040324003c04000095
:020000040000fa
:040328003c04000091
:020000040000fa
:04032c003c0400008d
:020000040000fa
:100400006f0921000eff24000e018800000000008b
:10041000000020000000e000020032000001200087
:100420002002880014000700150107000000e0000a
:1004300003003a00005f22000100200002003700a4
:100440000000200001002000810f70000100320038
:100450000f000700000020000000e0000200320052
:100460000000020000000000182a02000000000046
:100470000040da000000fe00200020000000e00044
:1004800002003200100020009001880000000600e9
:10049000a1028800800478000000eb001f003700f4
:1004a000e284440054a0b4009905ba00e2844400f8
:1004b00054a0b4009906ba00e284440054a0b400e9
:1004c0000006eb00476fde00fd07b200ae018800ba
:1004d000636ce10003003a000ad801000000eb0061
:1004e0000e003700606ce10008003a00004deb00a0
:1004f0000a05e800020039003420ec000af0a000f0
:100500008b05e900f9ff3e00040037006168e10057
:10051000010032000086eb000b00070019c7ba008b
:100520001905ba000e04e00003003a000a00e000da
:10053000dbff3a0000000600fe07b200ae028800b2
:100540008a047800f5ff37000cd0a300e20f4d00bd
:100550001c00390089027800354dba000a05e80010
:10056000020039003420ec000af0a0008b05e900fd
:100570000f003200254dba000a05e80002003900dc
:100580003420ec000af0a0008b05e90008003200de
:100590000c00e0000600320015cdba000a05e800a4
:1005a000020039003420ec000af0a0008b05e900bd
:1005b0008984e80054a0b4000b00e000e2ff3a0098
:1005c000000006009902ba00055d78008b05e9007d
:1005d000f7ff3200c82ade00055d78008b05e900d0
:1005e000f3ff32000c00e000f1ff320019ddba0029
:1005f000eeff3700422f040000000000aa2f040085
:10060000000000001a1c0400000000006a2304001f
:1006100000000000d223040000000000ea230400d0
:1006200000000000561d04000000000032280400f5
:1006300000000000a428040000000000bc28040002
:1006400000000000741e040000000000dc2804000c
:10065000000000004e29040000000000662904008c
:10066000000000003600f800809fbe00829fbe00a0
:10067000849fbe00869fbe00000820002b16070046
:100680004f03be004f02be004f01be004f00be0030
:100690003600f900004006003600f800809fbe00da
:1006a000829fbe00849fbe00869fbe00000820007f
:1006b0001e1607004f03be004f02be004f01be00d2
:1006c0004f00be003600f900004006003600f8007a
:1006d000809fbe00829fbe00849fbe00869fbe009a
:1006e00000042000111607004f03be004f02be0099
:1006f0004f01be004f00be003600f900004006006a
:100700003600f800809fbe00829fbe00849fbe001e
:10071000869fbe0000022000041607004f03be00a3
:100720004f02be004f01be004f00be003600f90070
:10073000004006003600f800809fbe00829fbe0089
:10074000849fbe00869fbe0010002000f7150700a2
:100750004f03be004f02be004f01be004f00be005f
:100760003600f900004006003600f800809fbe0009
:10077000829fbe00849fbe00869fbe002000200096
:10078000ea1507004f03be004f02be004f01be0036
:100790004f00be003600f900004006003600f800a9
:1007a000809fbe00829fbe00849fbe00869fbe00c9
:1007b00040002000dd1507004f03be004f02be00c1
:1007c0004f01be004f00be003600f9000040060099
:1007d0003600f800809fbe00829fbe00849fbe004e
:1007e000869fbe0080002000d01507004f03be008a
:1007f0004f02be004f01be004f00be003600f900a0
:10080000004006003600f8003200f8003400f8001e
:1008100010002000a00188001000200000d0fe0081
:100820003e8ea800e00125001010a0001189820072
:10083000e088820001000100b18982008089820085
:1008400001000100518a8200208a8200010001001b
:100850000000000000000000000000000000000098
:100860000b88a9003e8ea9003400f9003200f9007f
:100870003600f900004006000040da000000fe00eb
:04088000000005006f
:020000040000fa
:100884001400fa00889fbe000004780010002000c5
:10089400d0b79f000000eb00e0b79f00f0b79f00c7
:1008a40080ef9f006000b80080bf9f0091bf9f0051
:1008b400a0bf9f00b1bf9f00c0bf9f00d1bf9f00da
:1008c4001800e00002003d001838a30014003a00ac
:1008d40098007800618060000004e0000d003a0098
:1008e4000000eb0010049800180090008000eb005a
:1008f400e90f5000e08f5800100036000000eb00b4
:10090400100498005fb097004f04be000080fa0006
:10091400000006001000200010049800f2ff3700c9
:100924001878a300f0ff320098007800618060001e
:100934000004e000f7ff3a00e9ff37000006010079
:1009440057013700340137001a0137000701370017
:100954007f00370044003700360037001e003700a0
:100964000100370060013700f810900028b89000ab
:10097400808f5000660332001880a000f8109000a9
:1009840028b89000808f5000ec013900f8109000d6
:1009940028b89000808f5000daff360028b8900005
:1009a400c81090000080400020bc9800a8b89000b7
:1009b40078109000808f5000d2ff3600f81090001d
:1009c40021bc98005fb097004f04be000080fa007d
:1009d40000000600cfff37001880a00078009000c8
:1009e400880890000001e80072049800810f50000c
:1009f400c4ff36008000200010049800080890000e
:100a04000000e8007004980028e891000004e00069
:100a1400bcff3200a00e2000080040009e13070017
:100a24005fb097004f04be000080fa00000006008b
:100a3400b8ff370068109000e20f5000d301320075
:100a440078b89000e8b8900020c1900021c09800c8
:100a5400c808de0030c1900031c09800700020004a
:100a640010049800a7ff37001880a00078b8900001
:100a7400104090000078a3000c033200e8189000a6
:100a840058109000808f5000760239000000eb006f
:100a9400e0b79f0018189000efb09700808f5000c7
:100aa4000e0031006fb09700f400b900000044005c
:100ab40010089100104090000078a3002601320035
:100ac4006fb097000000e800e0b79f00981890000e
:100ad4006fb09700808f5000f2ff3e000040eb00a3
:100ae40080ef9f0038109000c810900000804000f4
:100af40030149800b810900028b89000808f5000ef
:100b040080ff3600a8b890003114980078b890009f
:100b1400410f2000888040002061900021609800ef
:100b2400c808de00306190003160980068109000c1
:100b34000000e000c9ff320068109000e20f50008e
:100b440070ff3a0060002000100498006dff370029
:100b54001880a0000000eb0030149800e00320008f
:100b6400600c980078b890006102200088804000f2
:100b74002061900021609800c808de003061900078
:100b84003160980068189000301498006810900044
:100b9400e20f5000ca013200d818900018289000c3
:100ba400808f5000e4003200e81890003830900044
:100bb400808f5000e0003200983090006819900057
:100bc40038309000000051000100b80080bf9f0041
:100bd40091bf9f000fb897009fb8970028319000ed
:100be400700111000201e900030033008100d1000b
:100bf4000080d300fbff370080bf9f0091bf9f00a0
:100c0400f820900058199000182890000000510016
:100c14000100b800a0bf9f00b1bf9f002fb897008c
:100c2400bfb8970008299000700111000201e90083
:100c3400030033008100d1000080d300fbff3700a4
:100c4400a0bf9f00b1bf9f000fb997009fb9970045
:100c54002fb89700bfb89700800f5100818f5900bb
:100c6400040036002fb89700bfb8970080bf9f00dc
:100c740091bf9f002fb89700bfb89700e00f5000b6
:100c8400e08f5800ac003200789190000fb89700c4
:100c94009fb897000200b800c0bf9f00d1bf9f005b
:100ca4002fb99700bfb997004fba9700dfba9700e2
:100cb4000500090042aad8008000eb00c0bf9f00d5
:100cc400d1bf9f00681090000000e000c7003a0008
:100cd40058b990004fb89700dfb89700cf91de0065
:100ce400800f5100818f59007d02360058b8900062
:100cf400cf80de00c0bf9f00d1bf9f00b80191002c
:100d04004fba9700dfba970078b8900004017800d2
:100d14008000eb000300010078b89000a050900020
:100d24008180fb00305090004800dd00008070009e
:100d34004fb99700dfb997000208780078b890009f
:100d4400a05890008180fb00305890004800dd00de
:100d5400008070004fb99700dfb99700020878004f
:100d64005000200010049800e6fe37001880a00010
:100d740028009000b80090000001e80022049800c8
:100d8400810f5000dffe3600380090000000e800bc
:100d940020049800400020001848a300d8fe3a0020
:100da4005fb097004f04be000080fa000000060008
:100db400d8fe37001880a1001800e00003003d00b1
:100dc40018e8a3000100320018d0a00008e0910048
:100dd4000004e00031013a001800e000c9fe3d00c3
:100de40018d8a300c7fe32001818a300c5fe3200ad
:100df4001828a300c3fe32001878a300c1fe3a00ed
:100e04001848a300bffe320018d0a1003000200013
:100e140010049800bbfe37001880a000080078007a
:100e240039110700dfb0970001006000d0b79f00c0
:100e3400f8b89000114090000074a1009040980010
:100e44009800910078b890000100010078b89000f3
:100e5400205190000281fb00b0509000c808dd00d2
:100e64008100710078b8900000c190000281fb00fd
:100e740010c090004800dd0082087000508282009b
:100e8400e20f50001e01320028e891000004e00047
:100e9400b9003a00200020001004980099fe3700a1
:100ea4001880a0000000eb00200498007004980053
:100eb4001830a1001810a1001898a3009d0032005a
:100ec4001840a10028e891000004e000030032006b
:100ed400a00e2000080040009d1207001000200012
:100ee4001004980087fe370008007800a30f07005d
:100ef400dfb0970001006000d0b79f00f8b8900001
:100f0400114090000074a100904098006810900077
:100f1400e20f5000be003200380090000000e800ec
:100f240020049800080890000000e800700498006d
:100f340010002000eaff3700289890008000eb00a2
:100f4400c0bf9f00d1bf9f00681090000000e00068
:100f540026003a005eff37006fb09700f400b90036
:100f64000000440010089100a05090008180fb0014
:100f7400305090004800dd000080700010007800c0
:100f8400f0b79f006fb09700f400b9000000440070
:100f9400d00991007fb197006fb09700f400b900b9
:100fa40000004400100891008000eb0003000100e1
:100fb4006fb09700f400b90000004400900891005d
:100fc400114090000074a000904098006fb097000a
:100fd4000000e800e0b79f00981890006fb09700f9
:100fe400808f5000affe3e00bcfe370068109000ba
:100ff400e20f50005aff3a000000eb00e0b79f00f8
:1010040080828200efb09700808f500054ff31003f
:101014006fb09700f400b900000044007001910023
:101024004fb89700dfb89700cf91de00800f5100d2
:10103400818f59008b0136006fb09700f400b9001e
:101044000000440070009100cf80de00c0bf9f000c
:10105400d1bf9f006fb09700f400b90000004400b6
:10106400d00991004fba9700dfba97006fb097008c
:10107400f400b90000004400100891000401780055
:101084008000eb00030001006fb09700f400b9008a
:101094000000440010089100a05090008180fb00e3
:1010a400305090004800dd00008070004fb9970078
:1010b400dfb99700020878006fb09700f400b90018
:1010c4000000440010089100a05890008180fb00ab
:1010d400305890004800dd00008070000c003200a1
:1010e4006fb09700f400b9000000440010089100ac
:1010f400a05890008180fb00305890004800dd002b
:10110400008070004fb99700dfb99700020878009b
:101114006fb097000000e800e0b79f008182820072
:101124006fb09700808f5000b9ff3e005000200040
:101134000cff37001840a00062ff3700a8b89000e9
:10114400481090000080500020bc9800a8b890007f
:1011540078109000808f5000eafd310078109000e4
:1011640020bc98005fb097004f04be000080fa00d6
:1011740000000600e7fd3700a00e20000800400034
:10118400f31107002000200043ff37001880a0005f
:1011940078b89000a0c090008180fb0030c190001e
:1011a4004811dd0002817000f808900081004100c0
:1011b40020c1900021c09800c808de0030c1900012
:1011c40031c0980078b8900020c190000281fb00e3
:1011d400b0c09000c808dd008100710050392000c3
:1011e400808f5000c7fd36000000e80060bc980006
:1011f40078b89000e8b8900020c1900021c0980011
:10120400c808de0030c1900031c0980013fe3700da
:101214000000eb00e0b79f0018189000efb09700b3
:10122400808f50003cff31006fb09700f400b9008c
:101234000000440090089100114090000074a10047
:10124400904098006fb097000000e800e0b79f005e
:10125400981890006fb09700808f50002eff3600d2
:101264006fb09700f400b9000000440090089100aa
:10127400114090000074a100904098006fb0970056
:101284000000e800e0b79f00981890006fb0970046
:10129400808f5000e4ff3e001fff3700dd890a0005
:1012a40018000000000e2000080040005012070043
:1012b40080c46400dd090a0018000000c6fe37007f
:1012c400e808900061bc980078b89000e8b89000f5
:1012d40020c1900021c09800c808de0030c19000f1
:1012e40031c09800b810900058109000808f5000c2
:1012f40029fe3100581090003014980026fe370063
:101304000000eb00e0b79f0080828200efb09700fe
:10131400808f5000dcfe31006fb09700f400b900fc
:101324000000440090089100114090000074a10056
:10133400904098006fb09700f400b900000044009a
:10134400b00891006fb09700f400b90000004400a9
:1013540010089100010001006fb09700f400b9007b
:101364000000440010089100205190000281fb000d
:10137400b0509000c808dd00810071006fb0970084
:10138400f400b900000044001008910000c190006e
:101394000281fb0010c090004800dd00820870004c
:1013a4006fb097000000e800e0b79f0081828200e0
:1013b4006fb09700808f5000b3fe36006fb0970077
:1013c400f400b9000000440090089100114090001e
:1013d4000074a100904098006fb09700f400b90029
:1013e40000004400b00891006fb09700f400b90009
:1013f4000000440010089100010001006fb0970044
:10140400f400b9000000440010089100205190003d
:101414000281fb00b0509000c808dd00810071001b
:101424006fb09700f400b900000044001008910068
:1014340000c190000281fb0010c090004800dd0054
:10144400820870006fb097000000e800e0b79f00ca
:10145400818282006fb09700808f5000aeff3e0003
:1014640089fe37000000000010c0b30080ef9f0029
:101474000000eb00e0b79f0018189000efb0970051
:10148400808f50009bfd31006fb09700f400b900cd
:101494000000440010089100a05090008180fb00df
:1014a400305090004800dd000080700034003200ad
:1014b4006fb09700f400b9000000440010089100d8
:1014c400104090000048a3002d003a006fb0970030
:1014d400f400b9000000440090089100114090000d
:1014e4000074a100904098006fb09700f400b90018
:1014f4000000440010089100a05090008180fb007f
:10150400305090004800dd0000807000100078002a
:10151400f0b79f007fb0970070004000f0b79f00c5
:101524006fb09700f400b900000044001008910067
:10153400a05090008180fb00305090004800dd00f6
:1015440000807000ffb09700010878006fb097002a
:10155400f400b900000044001008910080c8900015
:101564008180fb0010c890004800dd0000807000fe
:101574007fb197000201d10001b3200001084100ae
:101584006fb09700f400b900000044001008910007
:10159400a05890008180fb00305890004800dd0086
:1015a40000807000270032006fb09700f400b9008b
:1015b4000000440010089100104090000048a3006f
:1015c400200032006fb09700f400b900000044001e
:1015d40090089100114090000074a1009040980080
:1015e4006fb09700f400b9000000440010089100a7
:1015f400a05890008180fb00305890004800dd0026
:101604000080700010007800f0b79f007fb0970052
:1016140070004000f0b79f006fb09700f400b9006d
:101624000000440010089100a05890008180fb0045
:10163400305890004800dd0000807000ffb0970033
:10164400010878006fb097000000e800e0b79f0041
:10165400981890006fb09700808f50008aff3e006a
:1016640024fd37006fb09700f400b9000000440077
:10167400000991004fb89700dfb897008001eb0094
:10168400800f5100818f590072fe31006fb09700b6
:10169400f400b90000004400000891008000eb0051
:1016a400c0bf9f00d1bf9f006afe370008007800ca
:1016b400a10f0700dfb0970001006000d0b79f00c2
:1016c400681090000000e00017003a00f8b890009d
:1016d400114090000074a0009040980005fd370070
:1016e40068b990004fb89700dfb897008001eb000d
:1016f400800f5100818f590080fd310068b890003f
:101704008000eb00c0bf9f00d1bf9f007bfd37006e
:101714001880a1005fb097004f04be000080fa005b
:10172400000006007bfc370068109000e20f5000b8
:10173400f0fc3a00f8b89000114090000074a0004a
:1017440090409800e818900058109000808f500046
:101754000300310010c0b30080ef9f00e5fc3700a8
:101764000000eb00e0b79f00981890006fb097005e
:10177400808f50000a0036006fb09700f400b90063
:101784000000440090089100114090000074a000f3
:10179400904098006fb097000000e800f1ff370018
:0c17a4000040eb0080ef9f00d2fc3700fb
:020000040000fa
:1017b000f6874700889fbe008a9fbe008c9fbe00b0
:1017c0008e1f780010002000f0af9f004a11250006
:1017d0000004eb00080d78001032200090888a0089
:1017e000e4004500a0c62f00800878006607450089
:1017f00060392000000f7800b8888a00e8044500ae
:10180000c01b2500800c78006a014500a3c121009f
:1018100003097800a336220013898a00233d2200a1
:1018200003898a00a33e220023898a0012017800de
:10183000f1b79f00020001001900780022c22000c9
:10184000a0419000224098004811de00b041900075
:1018500032409800190078001a017800fa0f200031
:1018600080499000024898004811de00904990009d
:1018700012489800190078004041900042c0b3001f
:1018800042409800d04190005840980019007800dc
:10189000e041900000c6eb006c409800f0419000e1
:1018a000fbc7b3007b40980019007800a049900066
:1018b00028489800b04990003848980019007800ee
:1018c0008051900008509800905190001850980056
:1018d00019007800c0499000424898005049900093
:1018e0005848980019007800604990006c489800aa
:1018f000704990007b489800190078006a81440084
:101900008a026100a0519000255098004812de0024
:10191000b051900034509800190078008059900020
:1019200008589800905990001858980019007800ad
:10193000c051900048509800d051900058509800e5
:1019400019007800e05190006c509800f051900020
:101950007b50980019007800fe8644008a8166005a
:10196000a3b79f00a0599000cfe397002758980095
:10197000c869de0093b79f00b0599000afe39700ad
:10198000375898001900780080619000086098002e
:10199000906190001860980019007800c05990007c
:1019a00048589800d059900058589800190078006d
:1019b000e05990006c589800f05990007b589800be
:1019c0001900780003f32f00898141000a83610028
:1019d000a063900026609800c819de003063900074
:1019e0003360980019007800ffb0970091007800ec
:1019f00080c1900001c09800c808de0090c190002e
:101a000011c09800190078009e007800a0c19000d5
:101a100021c09800c808de00b0c1900031c0980015
:101a200019007800c0c0900048c09800d0c0900055
:101a300058c0980019007800e0c0900068c0980075
:101a4000f0c0900078c098001900780080c890001d
:101a500008c8980090c8900018c89800190078002d
:101a6000a0c8900028c89800b0c8900038c8980056
:101a700019007800c0c8900048c89800d0c89000ed
:101a800058c8980019007800e0c8900068c898000d
:101a9000f0c8900078c8980019007800e1f32f0092
:101aa000898040008a81600000d3900003d09800b4
:101ab000c808de0090d1900011d09800190078007d
:101ac000c0d0900048d09800d0d0900058d0980056
:101ad00019007800e0d0900068d09800f0d0900015
:101ae00078d098001900780080d8900008d8980025
:101af00090d8900018d8980019007800a0d89000cd
:101b000028d89800b0d8900038d8980019007800ec
:101b1000c0e0900048e09800d0e0900058e09800c5
:101b200019007800e0e0900068e09800f0e0900094
:101b300078e098001900780080e8900008e89800a4
:101b400090e8900018e8980019007800a0e890004c
:101b500028e89800b0e8900038e8980099007800ec
:101b6000114090000074a100904098009900780006
:101b7000114090000054a100904098009900780016
:101b8000114090000044a100904098009900780016
:101b9000114090000064a100904098001900780066
:101ba0001004a100190078001014a1009900780019
:101bb000114090000034a100904098006e0747004b
:101bc00000782000000f7800e10320000109780070
:101bd000f0814400070a20008709780072814400e0
:101be0000058220000097800e400510000b32000f2
:101bf00080087800f484440080222500800c78005e
:101c00006403410067d52100070b78002783220079
:101c1000b7898a00478a2200a7898a00c78b2200d9
:101c2000c7898a0016037800f1b79f00e2b79f00ca
:101c3000d3b79f00c4b79f00b5b79f00060001004f
:101c400019007800e6c020008a03630087bf9f0068
:101c5000a04390008ff39700274098004833de00a0
:101c6000b043900036409800190078001e037800b9
:101c7000804b9000064898004833de00904b90005f
:101c80001648980019007800404390006ec0b300d9
:101c90004e4098005043900058409800190078003a
:101ca000604390006c409800704390007b40980027
:101cb00019007800204b900028489800304b900085
:101cc0003848980019007800005390000850980098
:101cd000105390001850980019007800404b900065
:101ce00048489800504b90005848980019007800d8
:101cf000604b900068489800704b900078489800be
:101d000019007800e63420008a03630087bf9f0033
:101d1000a05390008ff39700275098004833de00bf
:101d2000b05390003650980019007800005b900086
:101d300008589800105b9000185898001900780017
:101d400040539000485098005053900058509800cd
:101d500019007800605390006c5098007053900008
:101d60007b50980019007800205b9000285898005c
:101d7000305b90003858980019007800006390009c
:101d800008609800106390001860980019007800af
:101d9000405b900048589800505b9000585898005d
:101da00019007800605b90006c589800705b9000a0
:101db0007b5898001900780020639000bfb297000c
:101dc00025609800b06290004fb297003460980090
:101dd00019007800dfb197009301780000c29000ed
:101de00003c09800c819de0010c2900013c098000c
:101df000190078006fb1970012017800a0c190001f
:101e000022c098004811de00b0c1900032c0980096
:101e10001900780040c1900048c0980050c190005f
:101e200058c098001900780060c1900068c0980000
:101e300070c1900078c098001900780042352000e9
:101e40008a01610000ca900003c898004811de00b2
:101e500090c9900012c8980019007800ffb0970050
:101e60009100780020c9900021c89800c808de00c1
:101e700030c9900031c898001900780021f22f0075
:101e8000898040000a81600080d1900002d09800d3
:101e9000c808de0010d1900011d098001900780019
:101ea000c0d0900048d09800d0d0900058d0980072
:101eb00019007800e0d0900068d09800f0d0900031
:101ec00078d098001900780080d8900008d8980041
:101ed00090d8900018d8980019007800a0d89000e9
:101ee00028d89800b0d8900038d898001900780009
:101ef000c0e0900048e09800d0e0900058e09800e2
:101f000019007800e0e0900068e09800f0e09000b0
:101f100078e098001900780080e8900008e89800c0
:101f200090e8900018e8980019007800a0e8900068
:101f300028e89800b0e8900038e898009900780008
:101f4000114090000074a100904098009900780022
:101f5000114090000054a100904098009900780032
:101f6000114090000044a100904098009900780032
:101f7000114090000064a100904098001900780082
:101f80001004a100190078001014a1009900780035
:101f9000114090000034a10090409800ec80440073
:101fa0000078200080087800e3032000830e78008a
:101fb000f0814400070a20008709780072814400fc
:101fc0000058220000097800e486460000af200097
:101fd000800e7800f484440040292500800c7800ad
:101fe0006a82400045e72100050a7800c58d22007d
:101ff000558a8a00e5942200458a8a006596220067
:10200000658a8a0014027800f1b79f00e2b79f004a
:10201000d3b79f00040001001900780004c120001c
:102020008a02620020439000254098004822de008a
:10203000b04290003440980019007800ffb097003b
:1020400091007800004a900001489800c808de001e
:10205000104a90001148980019007800c040900084
:102060004e409800d04090005840980019007800e9
:10207000e04090006c409800f04090007b40980059
:1020800019007800a048900028489800b0489000b7
:102090003848980019007800805090000850980047
:1020a000905090001850980019007800c048900097
:1020b00048489800d0489000584898001900780087
:1020c000e048900068489800f048900078489800f0
:1020d00019007800013f20000a826000a0529000a1
:1020e00024509800c808de0030529000315098000b
:1020f0001900780080589000085898009058900077
:102100001858980019007800c05090004850980066
:10211000d05090005850980019007800e05090007e
:102120006c509800f05090007b5098001900780097
:10213000a058900028589800b0589000385898003f
:10214000190078008060900008609800906090000e
:102150001860980019007800c058900048589800fe
:10216000d05890005858980019007800e058900016
:102170006c589800f05890007b589800190078002f
:10218000a0609000cfe0970021609800b0609000c0
:10219000afe397003760980019007800dfb197002f
:1021a0009300780080c1900001c09800c808de004c
:1021b00090c1900011c09800190078006fb197008d
:1021c0009200780020c1900021c09800c808de006d
:1021d00030c1900031c0980019007800c0c0900054
:1021e00048c09800d0c0900058c0980019007800ee
:1021f000e0c0900068c09800f0c0900078c09800df
:1022000019007800613f20000a81600080c99000b9
:1022100002c89800c808de0010c9900011c89800d4
:10222000190078009d00780020c9900021c898000e
:10223000c808de0030c9900031c898001900780045
:1022400001f12f00898040000a85600000d19000d4
:102250000ad09800c808de0010d1900011d0980074
:1022600019007800c0d0900048d09800d0d09000dd
:1022700058d0980019007800e0d0900068d09800fd
:10228000f0d0900078d098001900780080d89000a5
:1022900008d8980090d8900018d8980019007800b5
:1022a000a0d8900028d89800b0d8900038d89800ce
:1022b00019007800c0e0900048e09800d0e090005d
:1022c00058e0980019007800e0e0900068e098007d
:1022d000f0e0900078e098001900780080e8900025
:1022e00008e8980090e8900018e898001900780035
:1022f000a0e8900028e89800b0e8900038e898003e
:1023000099007800114090000074a100904098005e
:1023100099007800114090000054a100904098006e
:1023200099007800114090000044a100904098006e
:1023300099007800114090000064a100904098003e
:10234000190078001004a100190078001014a100f1
:1023500099007800114090000034a100904098004e
:102360007fa897004f0778004f06be004f05be00bc
:0c2370004f04be006f01b1000000060029
:020000040000fa
:10237c000800fa00889fbe008a1f78008c1f780026
:10238c001100200081bf9f008000eb0091bf9f00d7
:10239c0091bf9f00101990009fb89700810f5100ba
:1023ac0038013600a63220000836200006045400fe
:1023bc000884d100c7e1200005e020001fb9970078
:1023cc00fe11b90082004000a1909000a1bf9f00b7
:1023dc001fb99700fe11b90082004000b190900027
:1023ec00b1bf9f00bfb89700058153008191b90020
:1023fc00028142002fba97000402d0000482e90047
:10240c0088a2b90084004300624290000482fb0061
:10241c00f2419000c819dd00830172001fba9700c9
:10242c00fe22b90004024000c49490001400200065
:10243c008924dd008984ea0083846400e2419000f1
:10244c008041eb0069419800c84cde007245900059
:10245c0079419800624690000c86fb007245900012
:10246c004855dd000a0576001fbe9700fe66b900d0
:10247c008c044000d99490008924dd008984ea0002
:10248c008a8464006245900069419800c84cde0063
:10249c007245900079419800224690000c86fb0012
:1024ac00324590004855dd000a0576001fbe9700a6
:1024bc00fe66b9008c044000c99490008924dd00ac
:1024cc008984ea008a84640022459000294198009e
:1024dc00c84cde00324590003941980022469000ed
:1024ec000c86fb00324590004855dd000a0576004d
:1024fc001fbe9700fe66b9008c044000d994900072
:10250c008924dd008984ea008a84640022459000d5
:10251c0029419800c84cde003245900039419800a2
:10252c00424e90000c86fb00524d90004855dd0049
:10253c000a0576001fbe9700fe66b9008c044000a9
:10254c00c99490008924dd0089047500424d9000e7
:10255c0049499800c84cde00524d900059499800ea
:10256c00424e90000c86fb00524d90004855dd0009
:10257c000a0576001fbe9700fe66b9008c04400069
:10258c00d99490008924dd0089047500424d900097
:10259c0049499800c84cde00524d900059499800aa
:1025ac00f0400a001188000021419000a3409800df
:1025bc0031419000b440980061419000e340980094
:1025cc007141900002c3b300f240980001499000a1
:1025dc008348980011499000934898002149900035
:1025ec0092c1b300a24898003149900092c0b30048
:1025fc00b24898004149900002c4b300c248980008
:10260c0051499000d448980021519000a350980053
:10261c0031519000b350980041519000c350980034
:10262c0051519000d350980061499000e3489800b4
:10263c0071499000f3489800015190008350980024
:10264c00115190009350980061519000e350980004
:10265c0071519000f35098000159900083589800e4
:10266c00115990009358980021599000a358980044
:10267c0031599000b358980041599000c3589800b4
:10268c0051599000d358980061599000e358980024
:10269c0071599000f35898000161900084c0b30008
:1026ac008460980011619000936098001fb99700a6
:1026bc00fe11b90002014000c26c9100e1c464003b
:1026cc0062002000824cdd00314190000264a100c8
:1026dc0009417100b240980021619000a3609800fc
:1026ec0031619000b36098001fb99700fe11b900da
:1026fc000201400022999000c1649000c2609800d1
:10270c004811de00d1649000d260980061619000a5
:10271c00e360980071619000f36098001fb9970016
:10272c00fe11b9000201400072919000816c900082
:10273c00826898004811de00916c900092689800b5
:10274c0021699000a368980031699000b3689800e3
:10275c0041699000c368980051699000d368980053
:10276c0061699000e368980071699000f3689800c3
:10277c001fb99700fe11b900020140005299900058
:10278c0081749000827098004811de009174900062
:10279c00927098001fb99700fe11b9000201400019
:1027ac0042999000a1749000a27098004811de002c
:1027bc00b1749000b27098001fb99700fe11b90067
:1027cc000201400062999000e15c9000e258980090
:1027dc004811de00f15c9000f25898000161900005
:1027ec008460980011619000936098001fb9970065
:1027fc000200e00029003a00314190000234a000b0
:10280c00b2409800b141900082cfb30082c1610008
:10281c000304a000b34098002142900003cfb30002
:10282c0083416200a3409800a149900002c161005d
:10283c003240b300a24898001fb99700fe11b900ae
:10284c000201400002999000e1699000e268980052
:10285c004811de00f1699000f26898004141900047
:10286c000234a000c24098009fb897008100e80095
:10287c0091bf9f00101990009fb89700810f5100d5
:10288c00cefe3e000fb897004f0678004f0578003b
:10289c004f04be000080fa00000006003141900099
:1028ac000234a100b24098003141900083cfb300b4
:1028bc00034161003240b300b240980021429000c5
:1028cc0002cfb300024162000204a000a2409800b3
:1028dc002149900083416100a34898001fb99700db
:1028ec00fe11b9000201400002999000e1699000cc
:1028fc00e26898004811de00f1699000f2689800d7
:10290c00414190000234a000c24098009fb897004b
:10291c008100e80091bf9f00101990009fb89700ac
:0c292c00810f5100a5fe3e00d6ff3700d1
:020000040000fa
:102938000600fa00889fbe008a1f78001000200059
:10294800b0bf9f008000eb00c1bf9f000040eb00bc
:10295800c0f79f00f08082000010a100f0808a007c
:10296800f08082000020a100f0808a00f0808200c0
:102978000030a100f0808a00f08082000040a100b1
:10298800f0808a00f08082000070a000f0808a0049
:10299800f08082000090a100f0808a00f080820020
:1029a80000e0a000f0808a00f080820000f0a10022
:1029b800f0808a00000225000008eb0020002000bb
:1029c80050828a00e203200072828a0012322000bc
:1029d80062828a0080828a00c1bf9f008182820051
:1029e8004fb89700808f5000090036002205250057
:1029f8000009eb004fb897000000e800c0bf9f0037
:102a0800818282004fb89700808f5000f8ff3e0007
:102a1800600525000008eb00640040000008eb009a
:102a28000080e9000008eb00640040000008eb00ab
:102a38001000200010868a0020868a00e10020000d
:102a480031868a00f100200041868a00a10c250009
:102a58008048780009e8230069868a0008f4210084
:102a680078868a00030a200093868a0083868a0073
:102a780005582200a5868a0082022000b2868a00b4
:102a8800c2868a00041e2000d4868a00f480400092
:102a98008008eb00e0868a004100200001878a0058
:102aa80010878a006700200027878a0056002000c8
:102ab80036878a008a0e2500004d780059878a00db
:102ac80068878a0083878a0073878a0095878a00c7
:102ad800a2878a00b2878a00c4878a0074014500e9
:102ae8000009eb00d0878a00760145000049eb0019
:102af8006a0141000049eb00a3f62f0082814100e2
:102b080080497800c0f79f00b4c0b3000209b10043
:102b18000449780082c0b30067824100024a780005
:102b280024c22000a4838a0068824100014a7800f8
:102b38006b824100004aeb000482e900cff2970063
:102b4800054a780000024200cff29700054a780053
:102b580063024200004aeb000402e900004aeb006d
:102b6800f4ff270004848a0011848a00f28241005d
:102b7800800aeb0093417800e1c261008082620024
:102b8800c92add00e37080000390a10083817200f0
:102b9800e370880065f72f008a824200804a780037
:102ba800a3c0b30007844200034c78006784420046
:102bb800024c780008c2200008838a00688442001a
:102bc800014c78006b844200004ceb000884e9005b
:102bd800004ceb0000044400004ceb00630444008c
:102be800004ceb000804e900004ceb0064838a0009
:102bf80071838a0007044400000ceb0095427800ba
:102c080061c46200000464004844dd00e57080008f
:102c18000580a10085027400e5708800e5f92f00a1
:102c28008a824200804a780007844200004c78007b
:102c380067844200004c7800e8c0200048848a007d
:102c480068844200014c7800eb8042008048eb0029
:102c5800e98042008048eb00808040008048eb001b
:102c6800e38040008048eb008100e9008048eb00e9
:102c7800a4848a00b7848a0001782000c1848a006d
:102c88009542780061c26200000262004222dd00c3
:102c9800e17080000120a10081007200e1708800cd
:102ca800ec0044008048780025c0b300720244005c
:102cb800054a780073024400024a780004c12000e3
:102cc800e4848a0074024400034a780077024400ce
:102cd800004aeb000482e900004aeb0000024200cf
:102ce800004aeb0063024200004aeb000402e900dc
:102cf800004aeb009140780061c260000002620067
:102d08004722dd00e17080000170a100810072009f
:102d1800e170880001022000888040008048780027
:102d2800c0f79f0007824000064a7800678240008b
:102d3800024a780062c1200082858a0068814000ca
:102d4800034978006b8140000049eb000281e900eb
:102d58000049eb00000141000049eb00630141001c
:102d68000049eb000201e9000049eb0091407800be
:102d7800e1c0600000210a001c0e000081f62f004f
:102d8800828040008008eb00713e200021818a008b
:102d98002209b1000009eb000281e9000009eb00fb
:102da8007a0141000009eb0011828a008700410086
:102db8008008eb00318282000100e00001003a0047
:102dc80030828a008000eb00400425000008eb00f8
:102dd800d00d200040828a0050828200e20f50000d
:102de8000d003200c00225000008eb00f07c200036
:102df80070818a00200325000008eb0010322000b3
:102e080080818a003fb897004f0578004f04be00c4
:102e18000080fa0000000600b1818a00703e2000a0
:102e2800c0818a00e1818a00e08182000000e00020
:102e380002003a0010002000e0818a00e003200030
:102e4800d0818a00c00225000008eb00f07c200039
:102e580070818a00200325000008eb001032200052
:102e680080818a003fb897004f0578004f04be0064
:0c2e78000080fa0000000600e7ff3700b1
:020000040000fa
:102e84000400fa00889fbe008a1f780000047800be
:102e94000000eb00c0bf9f00800478000800e00041
:102ea400350032001800e00038003d002800900092
:102eb4008004eb000000e0002f0032003800900096
:102ec4000000e0002c003200480090000000e00008
:102ed40029003200580090000000e0002600320073
:102ee4001838a30035003a003c62ab0022003a00d7
:102ef4003c22ab0044003a00190020003e22ab0003
:102f04001d003a0020128000e0f79f0011800a00a3
:102f1400180000000004e00043003a0011c4b300ac
:102f24006ff19700814f51007600320030c4b30036
:102f3400eff0970080cf5000bb003200b0c4b30064
:102f44006ff19700804f5100c80032001900200033
:102f540040c5b300eff0970080cf500006003a0060
:102f64006ff19700425c98001810a0002914980093
:102f74002000200010049800090078004f05780014
:102f84004f04be000080fa000000060029149800d7
:102f94001810a1001800a1001830a1001820a100e9
:102fa40019002000090078004f0578004f04be0086
:102fb4000080fa0000000600f4ff3700190020002a
:102fc4003ce2ab00ecff320028109000890f500067
:102fd400e9ff3a0080002000c0bf9f004fb897006f
:102fe400ef0f50000b003e004fb897000000440064
:102ff400404890000080fb00401288004fb89700c2
:103004000000e800f4ff37003c22a900190020006a
:10301400e4ff37001830a1000000eb0020149800f2
:1030240019002000dfff3700281090000000440042
:10303400eff0970041589800281090000000e80035
:10304400201498002810900019002000e30f50006d
:10305400c9ff36001810a1000005eb002a149800df
:1030640000302500750b07008860900078589000a8
:1030740080cf5000c0ff3a0058589000e8589000a4
:10308400c808dd000080fb00008040001014980098
:1030940048599000424c980018109000504c9800e9
:1030a400181090004800de00604c980000c3b30084
:1030b400704c98000054980010c6b3001054980047
:1030c40000c0e80020549800684040003054980044
:1030d400cabf9f004fb89700e70f50004b003e0057
:1030e4004fb8970000004400404890000080fb0067
:1030f400401288004fb897000000e800c0bf9f004e
:10310400f4ff3700a800900091007800414c98002b
:10311400a800900091007800c808de00514c980087
:10312400b800900091007800614c9800b8009000bd
:1031340091007800c808de00714c9800c800900027
:103144009100780001549800c80090009100780024
:10315400c808de0011549800d8009000910078004f
:1031640021549800d800900091007800c808de002f
:10317400315498004054980050549800605498007a
:1031840070549800005c9800105c9800205c9800d3
:10319400305c98001830a000291498000000eb005f
:1031a400c0bf9f004fb89700e70f500072ff3e006a
:1031b4004fb8970000004400404890000080fb0096
:1031c400401288004fb897000000e800c0bf9f007d
:1031d4004fb89700e70f500071ff3e004fb89700bb
:1031e40000004400404890000080fb00401288002a
:1031f4004fb897000000e800c0bf9f004fb8970089
:10320400e70f5000eaff360065ff37001800900012
:103214000000e00062ff3a001814900068828a00ff
:10322400190020005fff370060072000401288006b
:103234004822ef004822ef001900200049128800bc
:103244004822ef004822ef004822ef000900400026
:1032540040128800090078004f0578004f04be0032
:103264000080fa000000060048ff37006ff0970066
:10327400405c98001810a000190020002914980040
:0c3284000000eb00100498003bff370036
:020000040000fa
:103290000400fa000002780011002000f1bf9f0036
:1032a0001404e00048003200e4409000efcf5000ea
:1032b00049003e0054499000e44090000281fb0028
:1032c0008180fb008110dd0001007800d02bb70069
:1032d00024499000e44090000281fb008180fb00c3
:1032e0008110dd0001007800f02bb7001449900038
:1032f000e44090000281fb008180fb008110dd0032
:1033000001007800202bb700e4409000e7cf500088
:1033100050003e00e440900081c04000c1ff9f008b
:10332000e440900002b1200012417800c4489000af
:103330008180fb004ff897008081fb008308dd004f
:103340008140710002b120000149780002b12000e3
:1033500012417800b44990008381fb004ff8970038
:103360008080fb008100e8008118dd008140710051
:1033700002b1200001497800e44090008180fb0008
:1033800002b8200082804000044990008248780002
:10339000f4409000e1cf500057003200e1cf5000e0
:1033a0005c003900e2cf50006b003200e3cf5000e8
:1033b000620032008af0a800344890000004e00067
:1033c000010032008cf0a800ffb8970001007800df
:1033d0000080fa0000000600644190008000eb00cd
:1033e000ff4f5100f9ff3e0054499000e440900027
:1033f0000281fb008180fb00f08050008110dd0025
:1034000001007800d22bb70024499000e4409000de
:103410000281fb008180fb00f08050008110dd0004
:1034200001007800f22bb70014499000e4409000ae
:103430000281fb008180fb00f08050008110dd00e4
:1034400001007800222bb700e4409000e7cf500045
:10345000b0ff3600e4409000efcf5000340036005b
:10346000e4409000f7cf500042003e00e44090005e
:10347000f0c0500081c04000c1ff9f00e4409000b8
:1034800002b1200012417800c44890008180fb0006
:103490004ff897008081fb008308dd0081407100b8
:1034a00002b120000149780002b1200012417800e9
:1034b000b44990008381fb004ff897008080fb00a7
:1034c0008100e8008118dd008140710002b1200018
:1034d00001497800e44090008180fb0002b82000a0
:1034e000828040000449900082487800f4409000b7
:1034f000e1cf5000a9ff3a008a30a800344890007c
:103500000004e000b0ff32008c30a800ffb8970044
:10351000aeff37008a10a800344890000004e00095
:10352000a9ff32008c10a800ffb89700a7ff370052
:10353000e4409000e8c0500077ff37008a70a80090
:10354000344890000004e0009fff32008c70a80017
:10355000ffb897009dff37008a50a80034489000bc
:103560000004e00098ff32008c50a800ffb89700dc
:1035700096ff3700644190008000eb00ff4f510040
:1035800092ff3e00e4409000f8c0500062ff370018
:020000040000fa
:103590000400fa0012002000e2bf9f008000eb0050
:1035a000f1bf9f000000e000200032001000e000aa
:1035b00021003d00100190008000eb000200e000bf
:1035c0001a0032009000900011017800d0009000a5
:1035d00081006100f1bf9f00a00090000100e000a9
:1035e00007003200900090009100780020019000c8
:1035f0009280500001f0a7008100ea00f1bf9f0017
:10360000a8810a0010000000e38f50005b00320028
:1036100010003400e58f5000760032006b0035005a
:10362000e68f50002f0032008000eb000100780090
:103630000080fa0000000600610098001010a10050
:103640001000a100020078000080fa0000000600cf
:10365000f9ff3700e18f500052003200e28f500036
:10366000f1ff3a0070019000ffb89700810f510000
:103670006a0036001010a0001018a30024003200c9
:1036800010017800e10061000104e00020003a0030
:10369000e00090008100e800610098006001900067
:1036a00080089000810f5100090039001000a0002f
:1036b0008008900061009800b00090000100e000d8
:1036c000030032003000900000000100e0bf9f00c6
:1036d000efb89700010078000080fa0000000600b3
:1036e000d5ff370010099000ffb89700810f5100f7
:1036f000e0ff3e0070019000ffb89700810f51007d
:10370000dcff39001010a1001018a300dcff3a0004
:1037100010017800e10061000104e00013003200b4
:103720001018a30011003a00e00090008100e800aa
:103730006100980060019000a0089000810f510086
:10374000e3ff39001000a100a0089000610098007c
:10375000c00090000100e000ddff3200400090005a
:1037600000000100e0bf9f00d9ff37008000eb00a0
:1037700061009800efb89700d6ff37007001900005
:10378000ffb89700810f5100baff3200700190001e
:10379000ffb89700810f5100b7ff32001010a10051
:1037a000d9ff370070019000ffb89700810f5100da
:1037b000b0ff390010099000ffb89700810f510049
:1037c000adff36001010a100cfff37007001900050
:1037d000ffb89700810f5100a6ff3a0070019000da
:1037e000ffb89700810f5100a3ff3a001010a1000d
:1037f000c5ff370010099000ffb89700810f5100f6
:10380000c0ff310070019000ffb89700810f510098
:10381000bcff36001010a00097ff37001009900081
:10382000ffb89700810f510093ff31001010a100e5
:04383000b5ff3700a9
:020000040000fa
:103834000200fa00881f7800000478000000eb0002
:10384400e0bf9f00f0000a001800000060012100a2
:10385400c860900040649800c800de005861900081
:1038640051649800e8004000686190006164980029
:10387400c808de007861900071649800010025009a
:1038840008699000016c9800c808de00186990006f
:10389400116c98004100250028699000216c980063
:1038a400c808de0038699000316c980021848000db
:1038b4006871900061749800c808de007871900007
:1038c400717498009180800008799000017c9800c0
:1038d400c808de0018799000117c980031848000bb
:1038e40028799000217c9800c808de00387990007f
:1038f400317c980081808000487190004174980068
:10390400c808de005871900051749800018080004e
:1039140048699000416c9800c808de00586990001e
:10392400516c98001180800068699000616c980067
:10393400c808de0078699000716c980021808000ce
:103944000871900001749800c808de001871900096
:1039540011749800318080002871900021749800bf
:10396400c808de0038719000317498008000eb00c4
:10397400e1bf9f00486990000281fb00d868900075
:10398400c808dd00810071006fb99700828f500074
:103994001400360083002100efb897006fb9970038
:1039a4004211dd0002814100c208dd0081004000b7
:1039b400b2187800a2107800efb897008100e800f0
:1039c400e1bf9f00486990000281fb00d868900025
:1039d400c808dd00810071006fb99700828f500024
:1039e400edff3e008000eb00e1bf9f00686990009e
:1039f4000281fb00f8689000c808dd0081007100b6
:103a04006fb99700828f500015003600c33325002c
:103a1400efb897006fb997004211dd0002814100b1
:103a24008180e800c208dd0081004000b2187800ff
:103a3400a2107800efb897008100e800e1bf9f0072
:103a4400686990000281fb00f8689000c808dd00f6
:103a5400810071006fb99700828f5000ecff3e0027
:103a6400c01b25004e030700a0808000e87890006a
:103a7400607c98004800de00f8789000707c980024
:103a840040848000c8789000407c98004800de00a4
:103a9400d8789000507c9800100020004f047800e3
:083aa4000080fa00000006009a
:020000040000fa
:103aac000200fa008000eb00f1bf9f00f0010a0059
:103abc0010000000e103210040619000416098007b
:103acc004809de00d0619000526098006881400087
:103adc00e0619000626098004811de00f061900097
:103aec0072609800a200250080699000026898001e
:103afc004811de009069900012689800e2002500e1
:103b0c00a0699000226898004811de00b06990000e
:103b1c003268980072848000e071900062709800a6
:103b2c004811de00f071900072709800e281800004
:103b3c0080799000027898004811de00907990000e
:103b4c001278980082848000a079900022789800e6
:103b5c004811de00b079900032789800d281800054
:103b6c00c0719000427098004811de00d071900036
:103b7c005270980052818000c06990004268980091
:103b8c004811de00d0699000526898006281800074
:103b9c00e0699000626898004811de00f0699000be
:103bac007268980072818000807190000270980099
:103bbc004811de0090719000127098008281800094
:103bcc00a0719000227098004811de00b071900036
:103bdc00327098000001eb00f2bf9f00c0699000aa
:103bec008381fb00506990004811dd000281710057
:103bfc00ffb99700830f51001400360024032100f5
:103c0c007fb99700ffb99700c219dd00830142000c
:103c1c004211dd0002814000331978002311780035
:103c2c007fb997000201e800f2bf9f00c0699000c5
:103c3c008381fb00506990004811dd000281710006
:103c4c00ffb99700830f5100edff3e000001eb0020
:103c5c00f2bf9f00e06990008381fb0070699000c7
:103c6c004811dd0002817100ffb99700830f5100ec
:103c7c0015003600843425007fb99700ffb99700f2
:103c8c00c219dd00830142000281e8004211dd000f
:103c9c000281400033197800231178007fb9970016
:103cac000201e800f2bf9f00e06990008381fb00f5
:103cbc00706990004811dd0002817100ffb9970016
:103ccc00830f5100ecff3e00802225001b050700ee
:0c3cdc00100020000080fa00000006002c
:020000040000fa
:103ce8000200fa008000eb00f1bf9f00f0010a001b
:103cf80010000000610621004061900041609800ba
:103d08004809de00d0619000526098006881400048
:103d1800e0619000626098004811de00f061900058
:103d2800726098004201250080699000026898003e
:103d38004811de0090699000126898008201250001
:103d4800a0699000226898004811de00b0699000d0
:103d58003268980092848000e07190006270980048
:103d68004811de00f0719000727098002283800084
:103d780080799000027898004811de0090799000d0
:103d880012789800a2848000a07990002278980088
:103d98004811de00b07990003278980012838000d4
:103da800c0719000427098004811de00d0719000f8
:103db8005270980092828000c06990004268980012
:103dc8004811de00d069900052689800a2828000f5
:103dd800e0699000626898004811de00f069900080
:103de80072689800b282800080719000027098001a
:103df8004811de009071900012709800c282800015
:103e0800a0719000227098004811de00b0719000f7
:103e1800327098000001eb00f2bf9f00c06990006b
:103e28008381fb00506990004811dd000281710018
:103e3800ffb99700830f510014003600a405210034
:103e48007fb99700ffb99700c219dd0083014200ce
:103e58004211dd00028140003319780023117800f7
:103e68007fb997000201e800f2bf9f00c069900087
:103e78008381fb00506990004811dd0002817100c8
:103e8800ffb99700830f5100edff3e000001eb00e2
:103e9800f2bf9f00e06990008381fb007069900089
:103ea8004811dd0002817100ffb99700830f5100ae
:103eb80015003600443525007fb99700ffb99700f3
:103ec800c219dd00830142000281e8004211dd00d1
:103ed8000281400033197800231178007fb99700d8
:103ee8000201e800f2bf9f00e06990008381fb00b7
:103ef800706990004811dd0002817100ffb99700d8
:103f0800830f5100ecff3e0040292500e104070023
:0c3f1800100020000080fa0000000600ed
:020000040000fa
:103f24000600fa0010002000d0bf9f000000eb0044
:103f3400e0bf9f00f0bf9f0001618000c1828a0042
:103f44007160800091828a0081608000a1828a0071
:103f5400b1608000e1828a00e0bf9f00818282001c
:103f64006fb89700808f500010003600e2012500e2
:103f74006fb897007a004000000040000000410044
:103f8400900078007fb8970000804000f0bf9f0049
:103f94006fb897000000e800e0bf9f0081828200b4
:103fa4006fb89700808f5000f1ff3e007fb89700f4
:103fb400b0828a00c28282000000eb00f14c200033
:103fc400810f510005003600c282820010002000db
:103fd400a1f02000810f510024003e006100600028
:103fe400c300dd00f08082000030a100008070007a
:103ff400f0808a00748a8200208b8200d38b820036
:10400400828c8200318d82000400700003007000f5
:104014000200700081007000e1806000c708dd00cc
:10402400f08082000070a10000807000f0808a009f
:10403400e001250012f20700dfb8970001006000dc
:10404400d0bf9f007705070000818200e50f500074
:1040540025003e00d08b820000f0a100d08b8a00a6
:104064005fb897000080fa00000006000000eb0033
:1040740061006000c300dd00f08082000030a10018
:1040840000807000f0808a00748a8200208b820095
:10409400d38b8200828c8200318d820004007000f8
:1040a400030070000200700081007000e180600075
:1040b400c708dd00f08082000070a100008070005d
:1040c400f0808a00e0012500edf10700dfb89700d9
:1040d40001006000d0bf9f005205070000818200ec
:1040e400e50f5000dbff3600e0888200a0609000fe
:1040f4008180fb00306090004800dd00008070008b
:10410400f08b8a00e08882009040900077810a005a
:1041140001000000cf08dd00d08b820000f0a10078
:1041240000807000d08b8a005fb897000080fa008e
:0841340000000600cdff37007a
:020000040000fa
:10413c000200fa000000eb00f0bf9f000000270017
:10414c00840fb60021003200a10920008007200056
:10415c000001eb0053f82000804978008149780079
:10416c0082497800207c8000e007b2000000a000ab
:10417c00720520006104200043f82000814978007a
:10418c008249780080497800eca10a00840f000075
:10419c00a8a00a00840f000080cf50000600320057
:1041ac007fb897008000e800f1bf9f0071382100b4
:1041bc00810f5000f4ff36000000eb007138210035
:1041cc007fb99700810f51003b003e0000fc2f008f
:1041dc008c2fb600860fb6000000a000307c880043
:1041ec00800c2000b0200a00880f0000f0f82f008f
:1041fc008a0fb6000060a000507c880080ff2f0062
:10420c008a0fb6000000a000507c8800f0cf2f0071
:10421c008a2fb600a1092000120020008007200080
:10422c0053f8200080497800814978008249780051
:10423c00eca10a00840f0000a8a00a00840f000063
:10424c0080cf500022003200207c8000e007b200ba
:10425c000000a000720520006104200043f820003b
:10426c00814978008249780080497800eca10a00e5
:10427c00840f0000a8a00a00840f000080cf50001b
:10428c00060032007fb897008000e800f1bf9f0065
:10429c0071382100810f5000f4ff3600eca20a00a7
:1042ac00840f0000a8a10a00840f00000000eb009e
:1042bc00814f5100020032000080fa00000006001d
:1042cc00713821007fb99700810f5100faff3e0031
:1042dc0084efa80084afab0006003a007fb89700cb
:1042ec008000e800f1bf9f0071382100810f500061
:1042fc00f8ff36000000eb0084afab00eeff32009d
:10430c00713821007fb99700810f5100eaff3e0000
:10431c0033a00a00840f0000610010000080fa0036
:08432c0000000600e6ff370067
:020000040000fa
:104334000200fa0011002000f1bf9f00a52fa90080
:104344002be3a90061e3a90097e3a900cde3a90049
:1043540003e4a90039e4a9006fe4a900a5e4a900d5
:1043640031002000f0210a00000300002130200069
:10437400914078000263ef003130200091407800d2
:104384000363ef0041302000914078000463ef00a4
:1043940051302000914078000563ef006130200027
:1043a400914078000663ef0071302000914078005e
:1043b4000763ef0081302000914078000863ef002c
:1043c40091302000914078000963ef00a130200073
:1043d400914078000a63ef00b130200091407800ea
:1043e4000b63ef00c06891000104e0000800320094
:1043f40070909000a1302000914078000ae3b7004b
:104404004800de00b1302000914078000be3b70093
:104414000cc3bf000c63ef000dc3bf000d63ef00be
:104424000ec3bf000e63ef000fc3bf000f63ef00a6
:1044340010c3bf001063ef0011c3bf001163ef008e
:1044440012c3bf001263ef0013c3bf001363ef0076
:1044540014c3bf001463ef0015c3bf001563ef005e
:1044640016c3bf001663ef0017c3bf001763ef0046
:1044740018c3bf001863ef0019c3bf001963ef002e
:104484001ac3bf001a63ef001bc3bf001b63ef0016
:104494001cc3bf001c63ef001dc3bf001d63ef00fe
:1044a4001ec3bf001e63ef001fc3bf001f63ef00e6
:1044b40020c3bf002063ef0021c3bf002163ef00ce
:1044c40022c3bf002263ef0023c3bf002363ef00b6
:1044d40024c3bf002463ef0025c3bf002563ef009e
:1044e40026c3bf002663ef0027c3bf002763ef0086
:1044f40028c3bf002863ef0029c3bf002963ef006e
:0c4504007fb897000080fa00000006005d
:020000040000fa
:10451000889fbe0089052500898a8a008000eb00fb
:10452000918a8a000083eb00c68a8a00e71425007e
:10453000f58f2f00178062000090a000800b78009c
:10454000d18a8a00f04c2000e08a8a0024032000ef
:10455000f48a8a00f005b000008b8a00481f200012
:10456000188b8a0023f42200a38a8a00a2fa220070
:10457000b28a8a00401625001010a0001000a0008a
:1045800017f0a000398b8a00418b8a00768b8a0055
:10459000908362000780a00007087800818b8a0062
:1045a000b7f02000978b8a00a48b8a00e705b10042
:1045b000b78b8a00c88b8a00538b8a00628b8a0073
:1045c0001010a0001000a00010f0a0000980e8006a
:1045d000e08b8a006c805400f08b8a00268c8a0065
:1045e000a0172500908362000780a00007087800cc
:1045f000318c8a00448c8a00a70f2000578c8a00d7
:1046000027012000678c8a00873e2000778c8a0073
:10461000038c8a00128c8a001010a1001000a100e7
:1046200010f0a1000980e900908c8a00a18c8a001a
:10463000d68c8a0000192500908362000780a000b4
:1046400007087800e18c8a00d7622100f78c8a0085
:10465000048d8a003706b100178d8a00077d20007f
:10466000278d8a00b38c8a00c28c8a001010a000ab
:104670001000a00010f0a00064804400408d8a006b
:10468000518d8a00868d8a00601a25009082620012
:104690000580a00005087800918d8a0051632000f4
:1046a000a18d8a00b48d8a001104b100c18d8a00e9
:1046b000d78d8a00638d8a00728d8a001010a00049
:1046c0001000a00010f0a000100020004f04be0059
:0446d00000000600e0
:020000040000fa
:1046d40010f0a6002d003700201490004015900023
:1046e4008608c3008608c1001201c100301b900077
:1046f4000600c8001a039000260598000a039000db
:10470400160598001001900092007800002990008e
:104714000109780010119000928010002019900077
:104724008208dd0030149000010d78008688c300f3
:104734008688c1008688c1001281c100401b900098
:104744000680c8000000cb000400cd0010239000b8
:1047540016a0e60006027800002390001620e6006a
:1047640006027800100c9000040c7800500c9000a5
:10477400040c7800401590000a0390001605980078
:10478400040d7800d0230400000000001001900004
:1047940092007800002990000109780000000600ca
:1047a400801f7800401090000018eb000008eb0018
:1047b4004f007800801f7800501090000018eb0024
:1047c4000018eb000008eb004f0078000000060022
:1047d400801f7800811f7800501090000118780025
:1047e4000118780001087800cf0078004f007800a5
:1047f400801f7800821f7800401090000218780013
:10480400020878004f0178004f007800000006008d
:1048140010f0a6001a0037001001900092007800f2
:104824000029900001097800101190009280100076
:10483400201990008208dd00701b90006019900020
:10484400010278001301c1000200c8000400cd0079
:104854001023900016a0e6000602780000239000c2
:104864001620e60006027800100c9000040c780074
:10487400500c9000040c78004a240400000000004e
:10488400100190009200780000299000010978003e
:04489400000006001a
:020000040000fa
:104898000800fa0011002000c1bf9f008000eb0053
:1048a800d1bf9f00e1bf9f00f1bf9f00d1bf9f0014
:1048b80010199000dfb89700810f5100560036009c
:1048c800a432200005362000848252008582d1005f
:1048d8005fb99700fe11b90082004000a1909000d6
:1048e800f1bf9f007fb997000201d0000281e90063
:1048f8008591b90082004200e14190008381fb006c
:10490800714190004811dd0002817100030023000d
:1049180002817100e1419000e24098004811de00f8
:10492800f1419000f2409800814990008381fb009a
:10493800114990004811dd00028171008201780060
:10494800330fb200014b9000834898004811de00f5
:104958009149900092489800114190000274a0007b
:1049680092409800414190000234a000c240980053
:104978001181fb00914190000278a3000e003200e3
:104988000003e200060035006fb997008201e800d5
:10499800e3bf9f0073382100830f5100f8ff3600f2
:1049a800efb9970072382100828f51001d003e0038
:1049b80001c3ab001b003a00814990008381fb00d2
:1049c800114990004811dd0002817100c200b30056
:1049d80081499000824898004811de009149900072
:1049e800924898009140900077810a0001000000e9
:1049f8004fb9970082806000c1bf9f00dfb8970061
:104a08008100e800d1bf9f0010199000dfb897001f
:104a1800810f5100aeff3e004fb897000080fa00aa
:104a2800000006000000eb000080fa00000006000d
:044a3800fcff370048
:020000040000fa
:104a3c000200fa0012002000f2bf9f0090029000ca
:104a4c0003e02000c4e120000302520085a2b9005b
:104a5c0083004200b00190000300e0002e003a00f9
:104a6c00614290000482fb00f1419000c819dd0006
:104a7c0083017200200290000411dd000281ea0023
:104a8c0003016100e1419000e24098004811de0012
:104a9c00f1419000f2409800400190000200e000cb
:104aac002d003200214290000482fb00b1419000a5
:104abc00c819dd0083017200200190001400200051
:104acc000221dd0002817100a1419000a2409800fa
:104adc004811de00b1419000b24098001182fb00f9
:104aec0091419000c819dd008301720020019000f3
:104afc00100020000201dd000281ea0003016100c8
:104b0c00f0020a0011000000f0bf9f007fb8970070
:104b1c000080fa0000000600614290000482fb0055
:104b2c00f1419000c819dd00830172002002900051
:104b3c000411dd0002817100e1419000e240980017
:104b4c004811de00f1419000f240980040019000c5
:104b5c000200e000d3ff3a00214290000482fb00e7
:104b6c00b1419000c819dd00830172002001900052
:104b7c00140020000221dd000281ea000301610023
:104b8c00a1419000a24098004811de00b141900074
:104b9c00b24098001182fb0091419000c819dd00d1
:104bac008301720020019000100020000201dd0042
:104bbc000281ea0003016100f0020a00110000000a
:104bcc00f0bf9f007fb897000080fa00000006003d
:044bdc00d1ff3700ce
:020000040000fa
:104be0004e5100006e000000800000001e500000ca
:104bf00030010000800000007a1000000a00000070
:104c0000800000000053000026000000800000002b
:104c10008a10000004000000800000003c530000e7
:104c20000c00000082000000815700000018010005
:104c300000009800a9000000bc5100006c000000ba
:104c4000800000000010000016000000820000003c
:104c500002000300000200000300230078000000af
:104c6000de070000000300000200d6005400000030
:104c700084100000060000008000000016100000f4
:104c80001400000080000000005000000a00000036
:104c900080000000485300000c000000820000006b
:104ca0001c4700000069080000004d00c100000022
:104cb000285200006c000000800000002a10000054
:104cc0001400000082000000020003000002000047
:104cd0000300bd005800000044270000000300004e
:104ce000020000008e1000000400000080000000a0
:104cf0003e10000014000000800000000a50000078
:104d00000a00000080000000545300000c00000066
:104d1000820000001c4700000069080000004d00f0
:104d2000c1000000945200006c00000080000000f0
:104d30005210000014000000820000000200030076
:104d4000000200000300bd005800000044270000de
:104d500000030000020000009210000004000000a8
:104d600080000000661000001400000080000000b9
:104d7000145000000a000000800000000000000045
:020000040000fa
:104d80000600fa0011002000d1bf9f008000eb0058
:104d9000e1bf9f00f1bf9f00e1bf9f00101990008d
:104da000efb89700810f510051003600a332200068
:104db00004362000030252000482d1006fb997002c
:104dc000fe11b90082004000a1909000f1bf9f0049
:104dd0007fb997000201d0000281e9008491b900f7
:104de00082804100e14290008582fb007141900089
:104df0004811dd000281720005002300028172006b
:104e0000e1429000e24098004811de00f14290003b
:104e1000f2409800814a90008582fb001149900081
:104e20004811dd000281720082027800350fb20065
:104e3000014b9000854898004811de00914a90008f
:104e4000924898009182fb00114190004811dd00ca
:104e50000281720002f0a100f0020a0011000000bd
:104e60006fb99700fe11b90002014000229990002d
:104e7000c1629000c26098004811de00d1629000cb
:104e8000d2609800c14290008582fb0051419000a1
:104e90004811dd00028172000230a000c142900082
:104ea000c24098004811de00d1429000d2409800e4
:104eb0001141900001c8b300814061008180fb0076
:104ec0008100e900cf08de005fb9970082806000b2
:104ed000d1bf9f00efb897008100e800e1bf9f00bd
:104ee00010199000efb89700810f5100b3ff3e00fa
:0c4ef0005fb897000080fa000000060088
:020000040000fa
:104efc000200fa0010002000f0bf9f00a40fa900d0
:104f0c0001eba90001aba90000062000022bb700a1
:104f1c0002eba90005eba90005cba900058ba800a5
:104f2c0000702000042bb70003f82f0020588000dd
:104f3c00808061000110a00021588800a100200091
:104f4c0090210a00060b000007cba90007eba90073
:104f5c00f1ff210082b0200012896000098ba900aa
:104f6c00096ba900094ba900092ba900090ba90081
:104f7c0008eba90008cba90001fc2f0080b0200091
:104f8c0010886000f1ff230052588000828060007e
:104f9c0001f0a00051588800f10f2c00a0b02000a7
:104fac00108860000aeba9000a0ba9000a2ba900c3
:104fbc000c0ba9000c2ba900c1ff2f00e2b02000a4
:104fcc001289600031ff2f00e0b0200010886000d3
:104fdc0000eca900000ca900002ca90000f0200096
:104fec00022cb70002eca900020ca900022ca900ab
:104ffc008000eb0090210a00d80b000090210a00e1
:10500c00d40b00000230200002007800d62bb70031
:10501c00b05e8000808061000110a000b15e88004d
:10502c0001c0210001007800d62bb70002007800e7
:10503c00da2bb700d25e8000028061000010a00065
:10504c00d05e880001007800da2bb7007fb897009b
:08505c000080fa0000000600cc
:020000040000fa
:1050640010f0a60032003700201490004015900084
:105074008608c3008608c1001201c100301b9000dd
:105084000600c8001a039000260598000a03900041
:1050940016059800100190009200780000299000f5
:1050a4000109780040019000810011001011900066
:1050b40092801000201990008208dd0030149000c6
:1050c400010d78008688c3008688c1008688c100e7
:1050d4001281c100401b90000680c8000000cb0074
:1050e4000400cd001023900016a0e600060278000c
:1050f400002390001620e60006027800100c9000b1
:10510400040c780041a3de005024900008054300fd
:10511400402490000a0c7800401590000a03900087
:1051240016059800040d7800a22804000000000071
:105134001001900092007800002990000109780085
:1051440000000600801f7800401090000018eb005b
:105154000008eb004f007800801f7800501090008a
:105164000018eb000018eb000008eb004f0078007b
:1051740000000600801f7800811f78005010900006
:10518400011878000118780001087800cf00780031
:105194004f007800801f7800821f78004010900034
:1051a40002187800020878004f0178004f00780058
:1051b4000000060010f0a600320037002014900012
:1051c400401590008608c3008608c1001201c10082
:1051d400301b90000600c8001a03900026059800b2
:1051e4000a039000160598001001900092007800c0
:1051f400002990000109780040019000810011000d
:105204001011900092801000201990008208dd0097
:1052140030149000010d78008688c3008688c10090
:105224008688c1001281c100401b90000680c8001e
:105234000000cb000400cd001023900016a0e6006f
:1052440006027800002390001620e600060278008b
:10525400100c9000040c780041a3de005024900050
:1052640008054300402490000a0c78004015900083
:105274000a03900016059800040d78004c290400d8
:1052840000000000100190009200780000299000b6
:105294000109780000000600801f7800401090008b
:1052a4000018eb000008eb004f007800801f780026
:1052b400501090000018eb000018eb000008eb0001
:1052c4004f00780000000600801f7800811f7800de
:1052d4005010900001187800011878000108780037
:1052e400cf0078004f007800801f7800821f78007c
:1052f4004010900002187800020878004f017800ee
:085304004f00780000000600d4
:020000040000fa
:10530c000600fa0011002000d1bf9f008000eb00c6
:10531c00e1bf9f00e1bf9f0010199000efb897000c
:10532c00810f51003c003600a532200006362000cb
:10533c00050353000683d1006fb99700fe11b90025
:10534c0082004000a1909000f1bf9f007fb99700b0
:10535c000201d0000281e9008691b90082804200ee
:10536c00614190000281fb00714290004822dd00f7
:10537c00040271000300230004827100614190005b
:10538c000041eb00e44098004822de00f14390001d
:10539c00f440980041629000c26098005162900005
:1053ac00d2609800414290000482fb005141900071
:1053bc004811dd00020172000230a0004142900051
:1053cc00c24098004811de0051429000d240980033
:1053dc00614190000281fb00f1409000c808dd00a3
:1053ec0081007100838160008301ea00cf19de0027
:1053fc00dfb8970081816100d3bf9f00efb89700a1
:10540c008100e800e1bf9f0010199000efb89700f1
:10541c00810f5100c8ff3e005fb897000080fa0072
:04542c000000060076
:020000040000fa
:105430000400fa0010002000e0bf9f000000eb0015
:10544000f0bf9f003dfb0700efb897000100600030
:10545000e0bf9f00c2010700efb8970001006000a5
:10546000e0bf9f0062020700efb8970001006000f4
:10547000e0bf9f00a3000700efb8970001006000a5
:10548000e0bf9f003f020700efb8970001006000f7
:10549000e0bf9f005d010700efb8970001006000ca
:1054a000e0bf9f001afc0700efb897000100600002
:1054b000e0bf9f0083020700efb897000100600083
:1054c000e0bf9f00f0f82f004028b6000028a90098
:1054d0002028a90001e1a800000880004f00de009c
:1054e000efb8970001006000e0bf9f006fb8970021
:1054f0000000e00001003a000000fe000028ab00c0
:1055000006003a007fb897008000e800f1bf9f00d6
:10551000f1522700810f5000f8ff36000028a90043
:105520000000eb00f0bf9f007efa0700f6010700c5
:0c5530007302070000000000f0ff3700cd
:020000040000fa
:10553c000600fa0011002000d1bf9f008000eb0094
:10554c00e1bf9f00f1bf9f00e1bf9f0010199000c9
:10555c00efb89700810f51002d003600a4322000c7
:10556c0005362000848252008582d1006fb99700e5
:10557c00fe11b90082004000a1909000f1bf9f0085
:10558c007fb997000201d0000281e9008591b90032
:10559c0082004200414190000234a000c2409800b9
:1055ac00614190000281fb00f1419000c819dd00bf
:1055bc00830171004819de0061439000e3409800bc
:1055cc00f20cb200f1419000f24098006141900061
:1055dc00f1409000c808dd000200230082806000ca
:1055ec008100e900cf08de005fb99700828060007f
:1055fc00d1bf9f00efb897008100e800e1bf9f008a
:10560c0010199000efb89700810f5100d7ff3e00a2
:0c561c005fb897000080fa000000060054
:020000040000fa
:1056280000818200e20f50000100320000000600f5
:10563800f08082000048a300fcff3a00f08082005e
:105648000018a300f9ff32007a30ec00d083800004
:10565800e70f500020003600e0838000918282002e
:1056680000804000e083880000848000a1828200de
:105678000080400000848800e08380004300de0052
:10568800e0838800008480004300de0000848800f6
:1056980080898200e18380000049900001489800d9
:1056a800c808de001049900011489800208a82003e
:1056b800018480000049900001489800c808de0075
:1056c8001049900011489800f08082000040a00026
:1056d800f0808a0000000600e0838000918282004a
:1056e80000804000e083880000848000a18282005e
:0c56f800008040000084880000000600d4
:020000040000fa
:105704000200fa0010002000f0bf9f00062eef00f8
:1057140080002000107188003e2eef001070880079
:1057240051392000f170880071002000d171880087
:105734000070880050382000e0708800c171880033
:105744003e8ea9003a8ea9003eaea9003aaea90049
:10575400234ea9001f4ea9000000eb0051052000b4
:10576400b1468800a10a2000b1468800006888007c
:1057740000fc2f00860db6002002b300306c8800b8
:10578400f00f2c00216c8000010160000130220028
:1057940082807000216c8800820db6000080a00019
:1057a400106c880040c2b30028edb70000802000d0
:1057b40051052000b1468800a10a2000b1468800a6
:1057c400006888007fb897000080fa000000060097
:020000040000fa
:1057d4000200fa0010002000f0bf9f00e001250045
:1057e400d3fa0700ffb8970001006000f0bf9f00e4
:1057f400e0012500e0f20700ffb897000100600017
:10580400f0bf9f00bcfd0700ffb8970001006000d7
:10581400f0bf9f00200725009cf60700ffb8970003
:1058240001006000f0bf9f00e005250097f6070027
:10583400ffb8970001006000f0bf9f0060082500da
:1058440092f60700ffb8970001006000f0bf9f00c8
:10585400a00925008df60700ffb89700010060003d
:10586400f0bf9f00e00a250088f60700ffb8970004
:1058740001006000f0bf9f00e00125000101070066
:10588400ffb8970001006000f0bf9f007fb8970049
:085894000080fa00000006008c
:020000040000fa
:10589c000200fa0012002000f2bf9f00900290005c
:1058ac0003e02000c4e120000302520085a2b900ed
:1058bc0083004200b00190000300e00011003200b0
:1058cc00614290000482fb00f1419000c819dd0098
:1058dc0083017200200090000011dd000281ea00bb
:1058ec000301610061409000e24098004811de0025
:1058fc0071409000f24098007fb897000080fa0049
:10590c0000000600614290000482fb00f14190000f
:10591c00c819dd0083017200200090000011dd0029
:10592c000281710061409000e24098004811de0055
:10593c0071409000f24098007fb897000080fa0008
:08594c0000000600efff370028
:020000040000fa
:105954000200fa0012002000f2bf9f0090029000a3
:1059640003e02000c4e120000302520085a2b90034
:1059740083004200b00190000300e00010003200f8
:10598400614290000482fb00f1419000c819dd00df
:1059940083017200200090000011dd00028171007b
:1059a40061409000e24098004811de007140900090
:1059b400f24098007fb897000080fa0000000600cb
:1059c400614290000482fb00f1419000c819dd009f
:1059d40083017200200090000011dd000281ea00c2
:1059e4000301610061409000e24098004811de002c
:1059f40071409000f24098007fb897000080fa0050
:085a040000000600eeff370070
:020000040000fa
:105a0c000200fa0010002000f0bf9f00c7f307004f
:105a1c00ffb8970001006000f0bf9f0061ef070026
:105a2c00ffb8970001006000f0bf9f0066ff070001
:105a3c00ffb8970001006000f0bf9f00e001250057
:105a4c0092fb0700ffb8970001006000f0bf9f00b9
:105a5c007fb897000000e00003003200f080820065
:105a6c000020a000f0808a0010000700ffb897000b
:105a7c0001006000f0bf9f00f02ba80080ff2f00fa
:105a8c006e08b6005000b300704388000b88a90064
:105a9c002b88a800f080820000f0a000f0808a0023
:0c5aac007fb897000080fa0000000600a0
:020000040000fa
:105ab8000600fa0010002000d0bf9f000000eb0095
:105ac800e0bf9f00f0bf9f0001eba8008a10f8001c
:105ad800000cf900508480004800dd008a10b700ef
:105ae800f0bf9f00036080007fb997006fb89700f0
:105af8008000e800e1bf9f0071382100810f50004d
:105b08000a0036006fb997000000eb0071382100d9
:105b1800810f510003003e008a10f8000a0bf900bb
:105b28005fb897000080fa0000000600828f5100dd
:105b3800f4ff3200036080007fb997006fb89700c8
:105b48008000e800e1bf9f0071382100810f5000fc
:085b5800ecff3e00f5ff3700f1
:020000040000fa
:105b60000200fa000000eb00f0bf9f008fefa900d9
:105b7000f0cf2f00922fb60000fc2f008e0fb60042
:105b80000000a000707c8800d1072000b0210a002e
:105b9000900f0000f0f82f00920fb6000050a00008
:105ba000907c880080ff2f00920fb6000000a000bc
:105bb000907c88008f0fa8008fefa8000000eb00fa
:105bc0008e0fe20009003d008fcfab0006003a00c7
:105bd0007fb897008000e800f1bf9f007138210076
:105be000810f5000f8ff3600100020000080fa00fe
:045bf00000000600ab
:020000040000fa
:105bf4000200fa0011c0b300e1ff9f009001900081
:105c040001e02000c2e12000010151008391b900ac
:105c140001014100c24190008381fb005241900088
:105c24004811dd0002817100a000900013002000e3
:105c34008118dd008280600001f0a7008100ea0085
:105c44008100ea00cf08de00e1ff9f0030009000f1
:105c5400830f5000030032006ff897000080fa00b1
:105c640000000600eff897000180fb00008051005f
:105c7400e0ff9f006ff897000080fa000000060024
:045c8400f8ff3700ee
:020000040000fa
:105c88000200fa00881f7800000478001000200045
:105c9800e0bf9f0008e091000004e00010003a0017
:105ca80028e891000004e00004003a006fb897006b
:105cb8004f0478000080fa0000000600a00e2000c3
:105cc800080040005bfb0700e0bf9f006fb897002b
:105cd8004f0478000080fa0000000600f7ff370044
:105ce800000e20000800400052fb0700e0bf9f00a4
:105cf80028e891000004e000ecff3200efff3700d5
:020000040000fa
:105d08000200fa0010002000f0bf9f00e0142500f8
:105d18001df60700ffb8970001006000f0bf9f0064
:105d28004016250018f60700ffb89700010060002c
:105d3800f0bf9f00a017250013f60700ffb89700d3
:105d480001006000f0bf9f00001925000ef6070053
:105d5800ffb8970001006000f0bf9f00601a25009f
:105d680009f60700ffb8970001006000f0bf9f0028
:0c5d78007fb897000080fa0000000600d1
:020000040000fa
:105d84000200fa0010002000f0bf9f00000820006d
:105d9400c01188003a22ef003c22ef0020022700c5
:105da400f0118800b0a22000001288004222ef0007
:105db4004c22ef004e22ef005022ef005222ef005f
:105dc4005422ef005622ef005822ef005a22ef002f
:105dd4005c22ef0039e2a80038a2a8003882a800ab
:0c5de4007fb897000080fa000000060065
:020000040000fa
:105df00001e1a90001a1a9000181a9000161a90097
:105e00000141a900003020000021b70000e1a900f5
:105e1000f0fc2f000021b6000041a9000021a900dc
:105e20000421ef00f070220040088800f0f82f00f5
:105e30004028b6000028a9002028a900100005006d
:020000040000fa
:105e40000200fa008000eb00f1bf9f004059900073
:105e5000d0599000e05890008381fb000281fb0044
:105e6000028141008180fb0081004100f1bf9f0061
:105e7000ffb8970001609800100020000080fa0031
:045e80000000060018
:020000040000fa
:105e84000200fa00881f780018002000e8bf9f0075
:105e9400e00125001cfd0700efb897000100600039
:105ea400e0bf9f00e00125001070a00008818a0077
:105eb4006fb897004f0478000080fa0000000600d5
:020000040000fa
:105ec400a005250020988a000080e90030988a0007
:105ed4006600500040988a000080e80050988a00cc
:105ee400403225000008eb004002b1001010a10070
:0c5ef4001030a10010f0a000100005000c
:020000040000fa
:105f00000200fa0010002000f0bf9f0000302500c2
:105f1000dcf30700ffb8970001006000f0bf9f00ae
:0c5f20007fb897000080fa000000060027
:020000040000fa
:105f2c0050998a00c03225001008e80000000000db
:105f3c000000000000000000000000000000000055
:085f4c00000000000000060047
:020000040000fa
:105f54000200fa000000eb00f0bf9f0010002000d8
:105f640000818a00e001250010f0a0007fb89700ae
:085f74000080fa0000000600a5
:020000040000fa
:020000040005f5
:047e0000ffffff0081
:020000040000fa
:020000040005f5
:047e2000ffffff0061
:020000040000fa
:020000040005f5
:047e3000f8ffff0058
:020000040000fa
:020000040005f5
:047e38007bffff00cd
:020000040000fa
:020000040005f5
:047e4000ff7fff00c1
:020000040000fa
:020000040005f5
:047e4800ffffff0039
:020000040000fa
:020000040005f5
:047e5000deffff0052
:020000040000fa
:020000040005f5
:047e5800ffffff0029
:020000040000fa
:020000040005f5
:047e6000ffffff0021
:020000040000fa
:020000040005f5
:047e6800ffffff0019
:020000040000fa
:020000040005f5
:047e7000ffffff0011
:020000040000fa
:020000040005f5
:047e7800ffffff0009
:020000040000fa
:020000040005f5
:047e8000fffcff0004
:020000040000fa
:020000040005f5
:047e8800fcffff00fc
:020000040000fa
:020000040005f5
:047ff800ffffff0088
:00000001FF
